:100000000C94DF000C94030D0C942A0D0C94070142
:100010000C9407010C9407010C9407010C94070140
:100020000C9407010C9407010C9407010C94070130
:100030000C9407010C9407010C9407010C94070120
:100040000C94510D0C9407010C9407010C940701BA
:100050000C9407010C9407010C9407010C94070100
:100060000C9407010C940701000000080002010035
:100070000003040700000000000000000102040863
:100080001020408001020408102001020408102002
:10009000040404040404040402020202020203032E
:1000A00003030303000000002300260029000000D2
:1000B0000000250028002B0000000000240027007D
:1000C0002A0000407A10F35A00A0724E180900105E
:1000D000A5D4E80000E87648170000E40B540200BD
:1000E00000CA9A3B000000E1F505000080969800E8
:1000F000000040420F000000A08601000000102711
:1001000000000000E80300000000640000000000A0
:100110000A00000000000100000000002C76D888D2
:10012000DC674F0823DFC1DFAE59E1B1B796E5E3E5
:10013000E453C63AE651997696E8E6C28426EB89FE
:100140008C9B62ED407C6FFCEFBC9C9F40F2BAA59B
:100150006FA5F490055A2AF75C936B6CF9676DC133
:100160001BFCE0E40D47FEF520E6B500D0ED902E37
:100170000300943577050080841E080000204E0A95
:10018000000000C80C333333330F986E12831141D3
:10019000EF8D2114893BE65516CFFEE6DB18D1849E
:1001A0004B381BF77C1D901DA4BBE42420328472C5
:1001B0005E228100C9F124ECA1E53D27430B112407
:1001C0001FBECFEFD8E0DEBFCDBF11E0A0E0B1E0B1
:1001D000ECE0F9E202C005900D92A83CB107D9F716
:1001E00022E0A8ECB1E001C01D92A032B207E1F715
:1001F00011E0CEEBD1E004C02297FE010E94E41191
:10020000CC3BD107C9F70E94F40F0C9484140C94D2
:1002100000000F931F93CF93DF9300D000D0CDB792
:10022000DEB78091E201882309F493C08091000138
:10023000909101010E94D60E892B61F080910901F5
:1002400090E00A9724F4809109018F5F0CC010920E
:1002500009010BC080910901882321F080910901D7
:10026000815001C08AE080930901E091090184E096
:10027000E89FF0011124E65FFE4F80819181A28109
:10028000B3818093F3019093F401A093F501B093AF
:10029000F60188EC91E00E94EB0B69E871E088ECD4
:1002A00091E00E943D0F40E065E088EC91E00E9403
:1002B000F20B809109018630C8F44091F30150910E
:1002C000F4016091F5017091F6012AE030E088ECCC
:1002D00091E00E94950F80910901882309F48DC057
:1002E00080910901813009F0B9C087C06091F301A4
:1002F0007091F4018091F5019091F6012091050132
:1003000030910601409107015091080129833A83F9
:100310004B835C830E949E1029813A814B815C81D2
:100320000E9408100E9470106093F2016091F20127
:100330004AE050E088EC91E00E94EC0F80910901C6
:10034000863009F4A0C080910901873009F062C0AD
:100350009AC080910001909101010E94D60E892BD4
:1003600031F140913A0150913B0160913C01709113
:100370003D0180913E0190913F01A0914001B091DB
:1003800041010091F3011091F4012091F5013091A8
:10039000F601800F911FA21FB31F481759076A0764
:1003A0007B070CF474C081E08093E10170C0809100
:1003B0003E0190913F01A0914001B0914101009117
:1003C000F3011091F4012091F5013091F601409173
:1003D0003601509137016091380170913901801BCD
:1003E000910BA20BB30B84179507A607B7070CF464
:1003F0004EC081E08093E0014AC086E08093F10125
:100400006091F10140E088EC91E00E94F20B6FE80E
:1004100071E018C0809109018830B9F1809109011B
:10042000893099F1809109018A3019F488E080932C
:10043000F1016091F10140E088EC91E00E94F20B43
:1004400063E971E088EC91E00F900F900F900F90AE
:10045000DF91CF911F910F910C943D0F8091090175
:10046000823041F080910901833021F080910901AF
:10047000843011F487E0C2CF80910901853009F002
:10048000BFCF88E0BBCF86E0D2CF87E0D0CF0F9040
:100490000F900F900F90DF91CF911F910F910895C2
:1004A0000C9418120C94201268EE73E080E090E037
:1004B0000E94BE0D20E042E060E188EC91E00E94E5
:1004C0000C0C88EC91E00E94EB0B40E060E088ECC3
:1004D00091E00C94F20B8091040160E00E94670EA1
:1004E0008091040161E00C94A00E0F931F93CF93B1
:1004F000DF9300D000D0CDB7DEB788EC91E00E944A
:10050000EB0B67E971E088EC91E00E943D0F40E061
:100510006DE088EC91E00E94F20B63E971E088ECF9
:1005200091E00E943D0F40E065E088EC91E00E9480
:10053000F20B6091F7017091F8018091F9019091AF
:10054000FA0103EE11E023E044E00E94F711B80144
:1005500088EC91E00E943D0F41E060E088EC91E082
:100560000E94F20B69E871E088EC91E00E943D0F77
:1005700041E065E088EC91E00E94F20B8091090176
:100580008630C0F44091F3015091F4016091F5017F
:100590007091F6012AE030E088EC91E00E94950F1E
:1005A000809109018823C1F180910901813009F00E
:1005B00072C032C06091F3017091F4018091F50135
:1005C0009091F601209105013091060140910701BB
:1005D0005091080129833A834B835C830E949E10CB
:1005E00029813A814B815C810E9408100E94701021
:1005F0006093F2016091F2014AE050E088EC91E0F2
:100600000E94EC0F80910901863009F459C0809155
:100610000901873071F454C086E08093F101609144
:10062000F10141E088EC91E00E94F20B6FE871E08B
:100630001AC080910901883009F444C080910901F1
:10064000893009F43FC0809109018A3019F488E0AB
:100650008093F1016091F10141E088EC91E00E940A
:10066000F20B63E971E088EC91E00E943D0F41E0FC
:100670006DE088EC91E00E94F20B6DE971E088EC8E
:1006800091E00F900F900F900F90DF91CF911F91FD
:100690000F910C943D0F80910901823079F0809187
:1006A0000901833059F080910901843039F080913B
:1006B0000901853009F0B3CF88E0AFCF87E0ADCF37
:1006C00086E0C6CF87E0C4CFCF92DF92EF92FF9251
:1006D000CF93DF93EC016A017B01642F0E945202E9
:1006E0009927F7FC9A958F2D7E2D6D2DCE010196C1
:1006F0000E945202B701992777FD9095892FCE016C
:1007000002960E9452026F2D772788279927CE01E3
:100710000396DF91CF91FF90EF90DF90CF900C94F4
:100720005202CF92DF92EF92FF920F931F93CF93DB
:100730006B017C01CB010E945002182FC60101966B
:100740000E945002C82FC60102960E945002082F34
:10075000C60103960E945002C82E8C2F90E0A0E0A4
:10076000B0E06627782F892F9A2F610F711D811DA8
:10077000911D10E020E030E0980111270027600F64
:10078000711F821F931FD12CE12CF12CFC2CEE2425
:10079000DD24CC246C0D7D1D8E1D9F1DCF911F91DE
:1007A0000F91FF90EF90DF90CF900895CF92DF925E
:1007B000EF92FF92CF93DF936B017C0160E0809119
:1007C00083010E94A00E60E0809184010E94A00E2F
:1007D000CFE1D0E0D701C6010C2E04C0B695A79595
:1007E000979587950A94D2F780FF02C061E001C017
:1007F00060E0809182010E94A00E61E080918301FF
:100800000E94A00E60E0809183010E94A00E2197BB
:1008100008F761E080918401DF91CF91FF90EF9024
:10082000DF90CF900C94A00E4F925F926F927F92C8
:100830008F929F92AF92BF92CF92DF92EF92FF92F0
:10084000CF93DF9300D000D0CDB7DEB780E89DE82E
:10085000ABE5B0E08093FF0190930002A09301020A
:10086000B093020280EC96ECADE2B0E08093FB0125
:100870009093FC01A093FD01B093FE0180913E0195
:1008800090913F01A0914001B0914101803C964C74
:10089000AD42B10570F080913E0190913F01A09171
:1008A0004001B091410181389D48AB45B10508F444
:1008B0002DC380EC96ECADE2B0E08093FF01909305
:1008C0000002A0930102B093020280E693EEA6E13B
:1008D000B0E08093FB019093FC01A093FD01B093E5
:1008E000FE0180913E0190913F01A0914001B091A5
:1008F00041018036934EA641B10570F080913E01D2
:1009000090913F01A0914001B0914101803C964CF3
:10091000AD42B10508F40FC380E693EEA6E1B0E066
:100920008093FF0190930002A0930102B093020212
:1009300080EB91E7ABE0B0E08093FB019093FC018A
:10094000A093FD01B093FE0180913E0190913F0183
:10095000A0914001B0914101803B9147AB40B1056E
:1009600070F080913E0190913F01A0914001B091C3
:1009700041018036934EA641B10508F4F5C280EBE3
:1009800091E7ABE0B0E08093FF0190930002A09369
:100990000102B093020288ED98EBA5E0B0E08093ED
:1009A000FB019093FC01A093FD01B093FE018091A7
:1009B0003E0190913F01A0914001B0914101883DDD
:1009C000984BA540B10570F080913E0190913F0198
:1009D000A0914001B0914101803B9147AB40B105EE
:1009E00008F4DBC288ED98EBA5E0B0E08093FF014E
:1009F00090930002A0930102B09302028CE69CED5A
:100A0000A2E0B0E08093FB019093FC01A093FD0174
:100A1000B093FE0180913E0190913F01A091400171
:100A2000B09141018C369C4DA240B10570F080918F
:100A30003E0190913F01A0914001B0914101883D5C
:100A4000984BA540B10508F4C1C28CE69CEDA2E02C
:100A5000B0E08093FF0190930002A0930102B09355
:100A6000020286E39EE6A1E0B0E08093FB01909352
:100A7000FC01A093FD01B093FE0180913E01909195
:100A80003F01A0914001B091410186339E46A140B3
:100A9000B10570F080913E0190913F01A09140011D
:100AA000B09141018C369C4DA240B10508F4A7C21B
:100AB00086E39EE6A1E0B0E08093FF019093000200
:100AC000A0930102B093020289E097EBA0E0B0E0AE
:100AD0008093FB019093FC01A093FD01B093FE0174
:100AE00080913E0190913F01A0914001B091410160
:100AF0008930974BA105B10570F080913E0190912E
:100B00003F01A0914001B091410186339E46A14032
:100B1000B10508F48DC289E097EBA0E0B0E08093C6
:100B2000FF0190930002A0930102B09302028CECAB
:100B30009BE5A0E0B0E08093FB019093FC01A093C3
:100B4000FD01B093FE0180913E0190913F01A09183
:100B50004001B09141018C3C9B45A105B10570F06D
:100B600080913E0190913F01A0914001B0914101DF
:100B70008930974BA105B10508F473C220913E015D
:100B800030913F01409140015091410180900B0212
:100B900090900C02A0900D02B0900E02C501B4011D
:100BA0000E94A51161387E4E8643910568F081E070
:100BB00090E0A0E0B0E08093030290930402A09341
:100BC0000502B093060208C01092030210920402BC
:100BD000109205021092060220913E0130913F01D1
:100BE0004091400150914101C0907A01D0907B0129
:100BF000E0907C01F0907D01C501B4010E94A51137
:100C0000A70196010E94B511CA01B9010E949C106A
:100C10000E94D9100E9470102B013C0160931302B6
:100C200070931402809315029093160220913E0156
:100C300030913F01409140015091410180917E01EE
:100C400090917F01A0918001B091810189839A8365
:100C5000AB83BC83C501B4010E94A5114B015C01AB
:100C6000A3019201C701B6010E94A511861A970A35
:100C7000A80AB90AA501940169817A818B819C81B6
:100C80000E94A511A70196010E94B51120930F02A1
:100C9000309310024093110250931202DA01C901FD
:100CA00063E0880F991FAA1FBB1F6A95D1F77FE0E9
:100CB000440C551C661C771C7A95D1F7842995291C
:100CC000A629B72980935A0190935B01A0935C01F8
:100CD000B0935D0189819A81AB81BC81E3E0880F8B
:100CE000991FAA1FBB1FEA95D1F781608093560117
:100CF00090935701A0935801B093590180917201CC
:100D000090917301A0917401B0917501F9E0880F81
:100D1000991FAA1FBB1FFA95D1F7409176015091F8
:100D2000770160917801709179012EE0440F551F91
:100D3000661F771F2A95D1F7842B952BA62BB72BEF
:100D4000826040916E0150916F01609170017091CD
:100D5000710136E0440F551F661F771F3A95D1F792
:100D6000842B952BA62BB72B809352019093530184
:100D7000A0935401B0935501409142015091430119
:100D8000609144017091450180916A0190916B01DD
:100D9000A0916C01B0916D01E7E1880F991FAA1F26
:100DA000BB1FEA95D1F7C0900702D0900802E090EF
:100DB0000902F0900A02F4E1CC0CDD1CEE1CFF1CD1
:100DC000FA95D1F78C299D29AE29BF2984609260BC
:100DD000C0906601D0906701E0906801F0906901D1
:100DE0002CE0CC0CDD1CEE1CFF1C2A95D1F78C29C5
:100DF0009D29AE29BF29C0906201D0906301E09087
:100E00006401F090650135E0CC0CDD1CEE1CFF1C8C
:100E10003A95D1F78C299D29AE29BF29C0905E0152
:100E2000D0905F01E0906001F0906101E3E0CC0CB4
:100E3000DD1CEE1CFF1CEA95D1F78C299D29AE29FB
:100E4000BF294E5F5F4F6F4F7F4FFDE1440F551F2E
:100E5000661F771FFA95D1F7842B952BA62BB72BFE
:100E600080934A0190934B01A0934C01B0934D01A4
:100E7000609146017091470180914801909149012C
:100E80000E94D60360914A0170914B0180914C0100
:100E900090914D010E94D60360914E0170914F01D7
:100EA00080915001909151010E94D60360915201AE
:100EB0007091530180915401909155010E94D60385
:100EC000609156017091570180915801909159019C
:100ED0000E94D60360915A0170915B0180915C0180
:100EE00090915D010F900F900F900F90DF91CF9137
:100EF000FF90EF90DF90CF90BF90AF909F908F903A
:100F00007F906F905F904F900C94D60310920702E1
:100F1000109208021092090210920A0281E090E0F9
:100F2000A0E0B0E080930B0290930C02A0930D021E
:100F3000B0930E02BECC81E090E0A0E0B0E08093E0
:100F4000070290930802A0930902B0930A0282E07C
:100F500090E0A0E0B0E080930B0290930C02A0938D
:100F60000D02B0930E02D8CC82E090E0A0E0B0E099
:100F70008093070290930802A0930902B0930A029B
:100F800084E090E0A0E0B0E080930B0290930C022C
:100F9000A0930D02B0930E02F2CC83E090E0A0E0AB
:100FA000B0E08093070290930802A0930902B093E7
:100FB0000A0288E090E0A0E0B0E080930B029093FA
:100FC0000C02A0930D02B0930E020CCD84E090E0D1
:100FD000A0E0B0E08093070290930802A09309027A
:100FE000B0930A0280E190E0A0E0B0E080930B02B1
:100FF00090930C02A0930D02B0930E0226CD85E0D3
:1010000090E0A0E0B0E08093070290930802A093E4
:101010000902B0930A0280E290E0A0E0B0E0809381
:101020000B0290930C02A0930D02B0930E0240CDE0
:1010300086E090E0A0E0B0E0809307029093080281
:10104000A0930902B0930A0280E490E0A0E0B0E02F
:1010500080930B0290930C02A0930D02B0930E02AA
:101060005ACD87E090E0A0E0B0E080930702909333
:101070000802A0930902B0930A0280E890E0A0E081
:10108000B0E080930B0290930C02A0930D02B093FA
:101090000E0274CDCF93DF9300D000D0CDB7DEB772
:1010A00061E0809184010E94670E61E0809184017B
:1010B0000E94A00E61E0809183010E94670E60E0B3
:1010C000809183010E94A00E61E0809182010E94C4
:1010D000670E60E0809182010E94A00E0E941404BD
:1010E000EE24E394A6E0DA2EB7E0CB2E18E0F12E42
:1010F000809104010E94D60E892B41F08091E1017C
:10110000811104C08091E001882391F380E00E9466
:10111000F10C809104010E94D60E892B09F0F4C0D5
:10112000E092E201809104010E94D60E892BA1F485
:101130008091ED019091EE01A091EF01B091F0014D
:101140000196A11DB11D8093ED019093EE01A09336
:10115000EF01B093F001E6CF8091ED019091EE01A7
:10116000A091EF01B091F001813A9648A140B105FC
:101170001CF140913E0150913F01609140017091FE
:10118000410180E090E00E9464036091090185E0E4
:1011900090E00E94520288EC91E00E94EB0B60EA22
:1011A00071E088EC91E00E943D0F68EE73E080E012
:1011B00090E00E94BE0D98C08CB3813009F48CBBC6
:1011C00042E050E069E071E080E00E94D10C88ECE0
:1011D00091E00E94EB0B69E871E088EC91E00E94DD
:1011E0003D0F40E065E088EC91E00E94F20B8091B9
:1011F00009018630C0F44091F3015091F4016091EF
:10120000F5017091F6012AE030E088EC91E00E944F
:10121000950F80910901882309F42BC18091090160
:101220008130A1F526C16091F3017091F4018091A4
:10123000F5019091F6012091050130910601409150
:1012400007015091080129833A834B835C830E94F4
:101250009E1029813A814B815C810E9408100E9476
:1012600070106093F2016091F2014AE050E088EC66
:1012700091E00E94EC0F80910901863009F4FFC0D3
:1012800080910901873009F006C1F9C080910901F8
:10129000823009F4F1C080910901833009F4ECC077
:1012A00080910901843009F4E7C0809109018530FB
:1012B00011F4F092F1016091F10140E088EC91E0CD
:1012C0000E94F20B6FE871E088EC91E00E943D0F04
:1012D000809104010E94D60E892BD1F780910401E0
:1012E0000E94D60E892BD1F380E00E94F10C10925F
:1012F000E2011092ED011092EE011092EF011092B6
:10130000F0010E947502A9C08091E1018823A9F033
:101310004091F3015091F4016091F5017091F60153
:1013200080913E0190913F01A0914001B091410117
:10133000840F951FA61FB71F18C08091E001882356
:10134000E1F04091F3015091F4016091F501709149
:10135000F60180913E0190913F01A0914001B09132
:101360004101841B950BA60BB70B80933E01909314
:101370003F01A0934001B09341011092E10110920E
:10138000E0010E94140460913E0170913F01809140
:101390004001909141012091050130910601409159
:1013A00007015091080129833A834B835C830E9493
:1013B0009E1029813A814B815C810E9408106093C4
:1013C000F7017093F8018093F9019093FA0160910D
:1013D000F7017091F8018091F9019091FA0120E0F4
:1013E00030E048EC52E40E94A11118160CF065C0E0
:1013F0006091F7017091F8018091F9019091FA01E3
:1014000020E030E04AE754E40E94041087FF55C012
:1014100040E06CE088EC91E00E94F20B61EB71E03F
:1014200088EC91E00E943D0F6091F7017091F80106
:101430008091F9019091FA0103EE11E023E044E07C
:101440000E94F71140E065E088EC91E00E94F20B09
:10145000B80188EC91E00E943D0F8CB3813009F413
:101460008CBB42E050E069E071E080E00E94D10C6A
:101470003FCED092F1011FCFC092F1011CCFD0928C
:10148000F1016091F10140E088EC91E00E94F20BE3
:1014900063E971E019CF80910901883059F080919A
:1014A0000901893039F0809109018A3051F7F092B1
:1014B000F101E7CFC092F101E4CF6091F7017091A3
:1014C000F8018091F9019091FA0120E030E048ECB8
:1014D00052E40E94041087FFA7CF40E06BE088EC45
:1014E00091E00E94F20B60EB71E09ACF88EC91E002
:1014F0000E94EB0B63EB71E088EC91E00C943D0FE4
:10150000CF93DF9300D000D0CDB7DEB760E070E0BE
:10151000CB010E94910360933E0170933F01809341
:1015200040019093410185E090E00E945002809339
:101530000901409136015091370160913801709155
:10154000390180913E0190913F01A0914001B091FD
:10155000410184179507A607B7070CF485C0409191
:101560003E0150913F016091400170914101809195
:101570003A0190913B01A0913C01B0913D0184174B
:101580009507A607B7070CF46FC0809109018091F9
:1015900009018B3008F068C0E091090184E0E89F00
:1015A000F0011124E65FFE4F80819181A281B38119
:1015B0008093F3019093F401A093F501B093F601A9
:1015C00060913E0170913F018091400190914101F5
:1015D00020910501309106014091070150910801C9
:1015E00029833A834B835C830E949E1029813A8130
:1015F0004B815C810E9408106093F7017093F801A1
:101600008093F9019093FA010E946B020E945402A8
:101610000E94760A68EE73E080E090E00E94BE0DC2
:101620000E94750242E050E069E071E080E00E94B3
:10163000D10C809102019091030160E00E94670E3D
:10164000809102019091030161E00E94A00E8091BF
:1016500000019091010162E00F900F900F900F90A8
:10166000DF91CF910C94670E8EED9BE8A4E0B0E083
:1016700080933E0190933F01A0934001B0934101BC
:101680001092090189CFCF92EF920F9309E0C02EFB
:1016900088E0E82E07E026E045E064E088EC91E091
:1016A0000E94AA0C0F91EF90CF900895CF93DF93F3
:1016B000EC0160E08E810E94A00E81E090E00E942B
:1016C000F80D61E08E810E94A00E81E090E00E9402
:1016D000F80D60E08E810E94A00E84E690E0DF911C
:1016E000CF910C94F80DEF92FF920F931F93CF932D
:1016F000DF938C01C0E0D0E0E62EF12CB7010C2E78
:1017000002C0759567950A94E2F76170F801EC0FD5
:10171000FD1F87810E94A00E2196C430D10571F76C
:10172000C801DF91CF911F910F91FF90EF900C9422
:10173000560BEF92FF920F931F93CF93DF938C0181
:10174000C0E0D0E0E62EF12CB7010C2E02C075955A
:1017500067950A94E2F76170F801EC0FFD1F87812D
:101760000E94A00E2196C830D10571F7C801DF9103
:10177000CF911F910F91FF90EF900C94560B1F93F8
:10178000CF93DF93EC01162F642F8C810E94A00E63
:101790008D818F3F19F060E00E94A00E8F85612F30
:1017A00084FF06C0CE01DF91CF911F910C94990B5D
:1017B00070E084E0759567958A95E1F7CE010E9407
:1017C000730B612FCE01DF91CF911F910C94730B9E
:1017D00040E00C94BF0B61E00E94E80B80ED97E0C5
:1017E0000C94F80D443008F043E0FC0123894217C3
:1017F00010F04FEF420FFC01E40FF11D2489260F7A
:101800002068622F0C94E80BFC016089262F24606D
:10181000208B6C600C94E80B0F931F93CF93DF9396
:10182000EC01423018F08F8588608F874B8B1C8AC3
:1018300080E48D8B6E8B70E0605C7F4F6F8B22231A
:1018400029F0413019F48F8584608F8761E08C81A5
:101850000E94670E8D818F3F19F061E00E94670E34
:1018600061E08E810E94670E00E010E08F8584FFAA
:1018700003C088E090E002C084E090E008171907F8
:1018800054F4FE01E00FF11F61E087810E94670EB2
:101890000F5F1F4FEBCF80E593EC0E94F80D60E0E7
:1018A0008C810E94A00E60E08E810E94A00E8D812E
:1018B0008F3F19F060E00E94A00E6F8564FD1DC08F
:1018C00063E0CE010E94730B84E991E10E94F80D60
:1018D00063E0CE010E94730B84E991E10E94F80D50
:1018E00063E0CE010E94730B86E990E00E94F80D40
:1018F00062E0CE010E94730B16C06062CE010E94AE
:10190000E80B84E991E10E94F80D6F856062CE01D9
:101910000E94E80B86E990E00E94F80D6F856062F6
:10192000CE010E94E80B6F856062CE010E94E80B39
:1019300084E0888BCE010E94040CCE010E94EB0B48
:1019400082E0898B66E0CE01DF91CF911F910F91EC
:101950000C94E80BCF92EF920F93FC01138212824A
:1019600083EC91E09183808364838FEF858346834A
:1019700027830087E186C28613861486158616861D
:10198000178620E041E060E1CF010F91EF90CF900A
:101990000C940C0C41E00E94BF0B81E090E0089594
:1019A00008958230E8F4E82FF0E0EE0FFF1FEB57C8
:1019B000FE4F71836083813041F0809169008C7F9C
:1019C000842B80936900E89A089580916900440F00
:1019D000551F440F551F837F842B80936900E99A1C
:1019E0000895823078F4813011F0E89801C0E998C8
:1019F000E82FF0E0EE0FFF1FEB57FE4F80ED9CE06D
:101A00009183808308951F920F920FB60F92112435
:101A10002F933F934F935F936F937F938F939F93F6
:101A2000AF93BF93EF93FF93E0918501F09186010F
:101A30000995FF91EF91BF91AF919F918F917F9108
:101A40006F915F914F913F912F910F900FBE0F902B
:101A50001F9018951F920F920FB60F9211242F937B
:101A60003F934F935F936F937F938F939F93AF9326
:101A7000BF93EF93FF93E0918701F091880109955F
:101A8000FF91EF91BF91AF919F918F917F916F9156
:101A90005F914F913F912F910F900FBE0F901F902C
:101AA00018951F920F920FB60F9211242F933F9308
:101AB0008F939F93AF93BF938091180290911902D7
:101AC000A0911A02B0911B023091170223E0230F5C
:101AD0002D3720F40196A11DB11D05C026E8230F66
:101AE0000296A11DB11D20931702809318029093B6
:101AF0001902A0931A02B0931B0280911C029091CC
:101B00001D02A0911E02B0911F020196A11DB11DE0
:101B100080931C0290931D02A0931E02B0931F029B
:101B2000BF91AF919F918F913F912F910F900FBED9
:101B30000F901F9018953FB7F89480911C029091D8
:101B40001D02A0911E02B0911F0226B5A89B05C0E0
:101B50002F3F19F00196A11DB11D3FBF6627782FB9
:101B6000892F9A2F620F711D811D911D42E0660F12
:101B7000771F881F991F4A95D1F708958F929F92DA
:101B8000AF92BF92CF92DF92EF92FF926B017C01F6
:101B90000E949B0D4B015C01C114D104E104F104CE
:101BA000F1F00E9403100E949B0D681979098A09BF
:101BB0009B09683E73408105910570F321E0C21ACC
:101BC000D108E108F10888EE880E83E0981EA11C78
:101BD000B11CC114D104E104F10429F7DDCFFF9059
:101BE000EF90DF90CF90BF90AF909F908F9008952F
:101BF0008230910538F0880F991F880F991F05973B
:101C00000197F1F70895789484B5826084BD84B516
:101C1000816084BD85B5826085BD85B5816085BDE7
:101C2000EEE6F0E0808181608083E1E8F0E0108200
:101C3000808182608083808181608083E0E8F0E041
:101C4000808181608083E1EBF0E08081846080832B
:101C5000E0EBF0E0808181608083EAE7F0E0808162
:101C600084608083808182608083808181608083C2
:101C70008081806880831092C1000895833081F054
:101C800028F4813099F08230A1F008958730A9F0CE
:101C90008830B9F08430D1F4809180008F7D03C00A
:101CA000809180008F7780938000089584B58F772E
:101CB00002C084B58F7D84BD08958091B0008F7778
:101CC00003C08091B0008F7D8093B0000895CF93C2
:101CD000DF9390E0FC01E458FF4F2491FC01E057B2
:101CE000FF4F8491882349F190E0880F991FFC01F0
:101CF000E854FF4FA591B49182559F4FFC01C591C7
:101D0000D4919FB7611108C0F8948C9120958223DB
:101D10008C93888182230AC0623051F4F8948C91AC
:101D2000322F309583238C938881822B888304C043
:101D3000F8948C91822B8C939FBFDF91CF91089563
:101D40000F931F93CF93DF931F92CDB7DEB7282F4A
:101D500030E0F901E859FF4F8491F901E458FF4F51
:101D60001491F901E057FF4F04910023C9F0882333
:101D700021F069830E943E0E6981E02FF0E0EE0FB2
:101D8000FF1FE255FF4FA591B4919FB7F8948C9136
:101D9000611103C01095812301C0812B8C939FBFDB
:101DA0000F90DF91CF911F910F910895CF93DF9303
:101DB000282F30E0F901E859FF4F8491F901E458E8
:101DC000FF4FD491F901E057FF4FC491CC2391F01C
:101DD00081110E943E0EEC2FF0E0EE0FFF1FEC553C
:101DE000FF4FA591B4912C912D2381E090E021F437
:101DF00080E002C080E090E0DF91CF910895CF9223
:101E0000DF92EF92FF920F931F93CF93DF937C01AA
:101E10006A01EB0100E010E00C151D0571F06991FD
:101E2000D701ED91FC910190F081E02DC70109955A
:101E3000892B19F00F5F1F4FEFCFC801DF91CF91B2
:101E40001F910F91FF90EF90DF90CF900895611553
:101E5000710581F0DB010D900020E9F7AD014150E3
:101E60005109461B570BDC01ED91FC910280F38177
:101E7000E02D099480E090E008950C94270FDC0198
:101E8000ED91FC910190F081E02D09948F929F9249
:101E9000AF92BF92DF92EF92FF920F931F93CF9377
:101EA000DF93CDB7DEB7A1970FB6F894DEBF0FBEB4
:101EB000CDBF7C01F42FD52ECB0119A2223008F41E
:101EC0002AE08E010F5D1F4F822E912CA12CB12C88
:101ED0006F2F7D2DA50194010E94B511F22FD32EF5
:101EE000CA01015011096A3014F4E0E301C0E7E3CC
:101EF000E60FD801EC93232B242B252B49F7B801AF
:101F0000C7010E94270FA1960FB6F894DEBF0FBE3F
:101F1000CDBFDF91CF911F910F91FF90EF90DF9098
:101F2000BF90AF909F908F900895CF92DF92EF92E5
:101F3000FF920F931F93CF93DF93EC016A017B0114
:101F40002115310579F4E881F9810190F081E02DC6
:101F5000642FDF91CF911F910F91FF90EF90DF9051
:101F6000CF9009942A303105E9F477FF1AC06DE269
:101F70000E943F0F8C0144275527BA014C195D0977
:101F80006E097F092AE0CE010E94460F800F911F43
:101F9000DF91CF911F910F91FF90EF90DF90CF9045
:101FA00008952AE0B701A601CE01DF91CF911F91DC
:101FB0000F91FF90EF90DF90CF900C94460F21157A
:101FC000310541F4DC01ED91FC910190F081E02DAF
:101FD000642F09940C94460F9A01462F50E060E05C
:101FE00070E00C94DF0F08950E94030E0E94F30F1F
:101FF0000E94800AC0E0D0E00E944A082097E1F3E6
:102000000E940000F9CF0895E7D008F481E0089518
:102010000CD046C13ED140F035D130F021F45F3FC5
:1020200019F0FEC0511187C12AC14BD198F39923F1
:10203000C9F35523B1F3951B550BBB27AA2762178C
:102040007307840738F09F5F5F4F220F331F441FD1
:10205000AA1FA9F333D00E2E3AF0E0E830D0915009
:102060005040E695001CCAF729D0FE2F27D0660FF6
:10207000771F881FBB1F261737074807AB07B0E835
:1020800009F0BB0B802DBF01FF2793585F4F2AF04B
:102090009E3F510568F0C4C04EC15F3FECF3983ECF
:1020A000DCF3869577956795B795F7959F5FC9F7A8
:1020B000880F911D9695879597F90895E1E0660F31
:1020C000771F881FBB1F621773078407BA0720F0AA
:1020D000621B730B840BBA0BEE1F88F7E095089513
:1020E000F8D088F09F5790F0B92F9927B751A0F0FA
:1020F000D1F0660F771F881F991F1AF0BA95C9F79C
:1021000012C0B13081F016D1B1E0089513C1672F2C
:10211000782F8827B85F39F0B93FCCF3869577954B
:102120006795B395D9F73EF4909580957095619534
:102130007F4F8F4F9F4F0895E89409C097FB3EF45F
:1021400090958095709561957F4F8F4F9F4F992304
:10215000A9F0F92F96E9BB279395F6958795779582
:102160006795B795F111F8CFFAF4BB0F11F460FF42
:102170001BC06F5F7F4F8F4F9F4F16C0882311F09A
:1021800096E911C0772321F09EE8872F762F05C0AE
:10219000662371F096E8862F70E060E02AF09A9549
:1021A000660F771F881FDAF7880F9695879597F93E
:1021B0000895A9D080F09F3740F491110EF0BBC074
:1021C00060E070E080E89FEB089526F41B16611D27
:1021D000711D811D2BC045C0990F0008550FAA0B1A
:1021E000E0E8FEEF16161706E807F907C0F012162A
:1021F0001306E407F50798F0621B730B840B950B2D
:1022000039F40A2661F0232B242B252B21F4089581
:102210000A2609F4A140A6958FEF811D811D08951E
:1022200097F99F6780E870E060E00895882371F473
:10223000772321F09850872B762F07C0662311F45F
:1022400099270DC09051862B70E060E02AF09A9596
:10225000660F771F881FDAF7880F9695879597F98D
:1022600008959F3F31F0915020F4879577956795B9
:10227000B795880F911D9695879597F908959FEFCB
:1022800080EC089500240A9416161706180609060D
:10229000089500240A9412161306140605060895DC
:1022A000092E0394000C11F4882352F0BB0F40F464
:1022B000BF2B11F460FF04C06F5F7F4F8F4F9F4FA4
:1022C000089557FD9058440F551F59F05F3F71F026
:1022D0004795880F97FB991F61F09F3F79F087958D
:1022E0000895121613061406551FF2CF4695F1DF16
:1022F00008C0161617061806991FF1CF86957105A6
:10230000610508940895E5DFA0F0BEE7B91788F4E9
:10231000BB279F3860F41616B11D672F782F8827CA
:10232000985FF7CF869577956795B11D9395963908
:10233000C8F30895E894BB2766277727CB0197F960
:1023400008954ADF08F48FEF0895DB018F939F9380
:102350000E94D711BF91AF91A29F800D911DA39FA5
:10236000900DB29F900D11240895A1E21A2EAA1B80
:10237000BB1BFD010DC0AA1FBB1FEE1FFF1FA21735
:10238000B307E407F50720F0A21BB30BE40BF50B32
:10239000661F771F881F991F1A9469F760957095BB
:1023A000809590959B01AC01BD01CF0108950E94DD
:1023B000E811A59F900DB49F900DA49F800D911DD5
:1023C00011240895EE0FFF1F0590F491E02D09945C
:1023D000A29FB001B39FC001A39F700D811D112466
:1023E000911DB29F700D811D1124911D0895EF92D2
:1023F0000F931F93CF93DF93E80147FF02C034E1AF
:1024000001C034E0E42FFF27E7FDF095F7FF03C09C
:10241000F195E195F109E32E022F2E2FAE010E94D6
:102420002E12CE01DF91CF911F910F91EF90089561
:10243000F999FECF92BD81BDF89A992780B508958C
:10244000262FF999FECF1FBA92BD81BD20BD0FB6D0
:10245000F894FA9AF99A0FBE019608956F927F92B6
:102460009F92AF92BF92CF92DF92EF92FF920F9323
:102470001F93CF93DF93CDB7DEB729970FB6F894AC
:10248000DEBF0FBECDBF6A01B22E102F0C3320F479
:10249000FF24F394F00E02C04CE3F42E0F2D27E03E
:1024A000AE014F5F5F4F0E94AC137981272F2970D7
:1024B000213031F0E1FC06C0E0FC06C060E005C060
:1024C0006DE203C06BE201C060E2AE2DA07173FF4C
:1024D00036C0662311F084E001C083E08B1510F450
:1024E000B81A01C0B12CA1110BC0F6018B2D90E2DE
:1024F000882319F091938150FBCFCB0CD11CB12CC8
:10250000662331F0F601608396012F5F3F4F69012A
:10251000C6010396E2FE05C02EE4F601208331E4F5
:1025200004C02EE6F601208331E631832283FC01CC
:102530002B2D30E22223F1F131932150FBCF72FF9A
:1025400040C0662311F084E001C083E08B1510F4D5
:10255000B81A01C0B12CA1110BC0F6018B2D90E26D
:10256000882319F091938150FBCFCB0CD11CB12C57
:10257000662331F0F601608396012F5F3F4F6901BA
:10258000C6010396E2FE07C029E4F60120832EE48B
:10259000218326E406C029E6F60120832EE6218366
:1025A00026E62283FC012B2D30E2222319F0319301
:1025B0002150FBCFFC01EB0DF11D10828EEF9FEF40
:1025C000B7C0B1E0611101C0B0E04B2F50E0181668
:1025D000190624F49C012F5F3F4F02C021E030E038
:1025E000240F351F112329F0412F50E04F5F5F4F1B
:1025F00002C040E050E0420F531F2B2D30E0421745
:10260000530714F4B41A01C0B12C2E2D287159F4BB
:10261000F6012B2D30E2222319F031932150FBCF0C
:10262000CB0CD11CB12CBB2331F0F6016083960199
:102630002F5F3F4F6901A1110BC0F6012B2D30E335
:10264000222319F031932150FBCFCB0CD11CB12C9C
:10265000F80E0A81372F3071A32E74FF03C00133A7
:1026600009F4FA941F142CF42F2D293018F028E0C7
:1026700001C021E0682F392F97FF02C060E030E0F1
:10268000462F532F612C712C3EE2932EBC01621B0E
:1026900071099B01DC01A41BB50BE1E0F0E0EC0F3C
:1026A000FD1FAE0FBF1FE12EF12CF194E194F10854
:1026B0004F3FFFEF5F0731F4F6019082B6016F5F85
:1026C0007F4F6B01841795074CF02417350734F4BE
:1026D000BD01660D771DFB01118101C010E3415062
:1026E0005109FFEF6F1A7F0AB6016F5F7F4F4E15DA
:1026F0005F0524F0F60110836B01DACF4817590704
:1027000039F4063320F4053319F4A11001C011E3A4
:10271000F6011083FB018B2D90E2882319F0919331
:102720008150FBCFFB01EB0DF11D108280E090E0AA
:1027300029960FB6F894DEBF0FBECDBFDF91CF91C3
:102740001F910F91FF90EF90DF90CF90BF90AF90CF
:102750009F907F906F900895283008F027E03327EE
:10276000DA01990F311D87FD9160009661057105B1
:1027700039F432602E5F3D9330E32A95E1F70895F6
:102780009F3F30F080387105610509F03C5F3C5F88
:102790003D93913008F08068911DDF93CF931F9394
:1027A0000F93FF92EF92192F987F9695E92F9695A8
:1027B0009695E90FFF27E45EFE4F99273327EE2415
:1027C000FF24A701E70105900894079428F4360F29
:1027D000E71EF81E491F511D660F771F881F991F9E
:1027E0000694A1F70590079428F4E70EF81E491FF8
:1027F000561FC11D770F881F991F661F0694A1F7EA
:102800000590079428F4F80E491F561FC71FD11DC5
:10281000880F991F661F771F0694A1F705900794EC
:1028200020F4490F561FC71FD81F990F661F771F27
:10283000881F0694A9F784911095177041F0D695DA
:10284000C79557954795F794E7941A95C1F7E2EC29
:10285000F0E06894159015913591659195910590EA
:102860007FE27395E118F10A430B560BC90BD009AF
:10287000C0F7E10CF11E431F561FC91FD01D7EF487
:10288000703311F48A95E6CFE894015030F0080FC8
:102890000AF40027021708F4202F2395022F7A3319
:1028A00028F079E37D932A95E9F710C07D932A9566
:1028B00089F6069497956795379517951794E118BB
:1028C000F10A430B560BC90BD00998F023957E9162
:1028D00073957A3308F070E37C932013B8F77E91F8
:1028E00070617D9330F0839571E37D9370E32A9559
:1028F000E1F71124EF90FF900F911F91CF91DF919D
:0C290000992787FD90950895F894FFCF6B
:10290C000A0002000E00007A4405010000000500D8
:10291C0000000A00000019000000320000006400F2
:10292C000000E8030000881300001027000050C3CB
:10293C000000A0860100D8590000A02E63007F8DF6
:10294C005B000100000005004001FC02D96133016D
:10295C000000425E0100A961032008D2A50003001B
:10296C00000001000000FF00000001000000010059
:10297C0000000F00000010000000350C0000350CAA
:10298C00000011100FD00CD00C535445503A006B72
:10299C00487A004D487A00465245513A004F4E0055
:1029AC00534156454420544F20454550524F4D00FD
:1029BC002020004D4158323837305F565F310000CF
:0829CC00000000CA0CFF0E0020
:00000001FF
